S107002A4F0002017C
S1230100CE05178D6C815926022003CE07038D615F81592604BD04F15CD72BCE07568D5191
S12301205F814E2702C602D72CCE07BA8D4381582702864F972ACE07D78D365F814E2701DD
S12301405CD72DBD0507C62ECE003CE700088C007D26F8CE4F58DF57CE584FDF5FCE02042C
S1230160DF34DF359726BD03FC7D002D27117E025CBD04F1BDC006811B26037E0367397D85
S1230180002B27028DEE962A88179729864097247F00277F00287F00257F003BCE0027BD8F
S12301A00387812E2638BD039B4D27327F0037BD0428D63927289627270481072602DB2C07
S12301C09628270481072602DB2CD1252206260EC501270A9639973BD725DE27DF227A0015
S12301E02427145F7C0028962881072303D7285C96271B972720A57D003B27537F0026960A
S1230200349B3B4C97349635903B97357C0036CE094FBD04F196228B31BDC00396238B4154
S1230220BDC003CE095CBD04F1CE003BBD04DACE096CBD04F1DE22DF277C0037BD0428BD5D
S123024003FC963527069636814026107E0300CE097EBD04F1962626F37C0026962A972961
S1230260CE07A3BD017181582605BD03FC20ED81382277803125739727BD01748148226A26
S1230280804125669728CE0027BD0387CE0777812E2617BD039BCE07F14D270E7F0037BDC5
S12302A004287D00392608CE082ABD04F120AD7F0026CE085DBD04F1CE0039BD04DACE08A9
S12302C06FBD04F196359B394C97359634903997347C00367C0037BD0428BD03FC963427E9
S12302E01F9636814027197E017FCE0999BD0171815926B9BD0507962626057C002620E75F
S1230300CE087EBD04F1CE0035BD04DACE0889BD04F1CE0034BD04DACE089DBD04F1CE088C
S1230320BF96359134273D220CCE08A7BD04F1D634D035200ACE08C7BD04F1D635D034CE44
S123034008D2BD04F1CE08DED1362718CE090BC1052311CE0900C10A230ACE08F8C10F23A7
S123036003CE08EDBD04F1CE0916BD0171814E2706BD05077E0146CE0939BD04F17EC0005B
S12303808D059629A70039A600E601484848CE003C1B2704084A26FCA6003996298817972B
S12303A0318608972ECE03ECDF2FD627A600270D2B075CC107222820045D27235AD720D681
S12303C028DE2FA601270D2B075CC107221120045D270C5AD721CE00208DAC9131270CDE80
S12303E02F0808DF2F7A002E26C04F390001FF01FF00FFFF00FF01FF01000101CE09C1BD41
S123040004F1CE003C86304C972EBDC003C6088620BDC003A600BDC003085A26F28D0696D5
S12304202E813826E27E05077D00372706CE0027BD03807F00398608972ECE03ECDF2FDE75
S12304402FA6009732A60197337F003896279720962897217F003A963227152B0B7C002059
S123046096208107225F20087D002027587A0020963327152B0B7C0021962181072246203C
S1230480087D0021273F7A0021CE0020BD038716962988171126107C003A7D003827B8CEA9
S12304A00020BD038020B0D129261A7D00382606963A9B3997397D0037270A7D00382605B4
S12304C07C0038208796308B02D62FC9009730D72F7A002E27037E043F39E6004F4CC00AB8
S12304E024FBCB0A4A27028D01178B307EC0038D23A60008815E260486108D11812F26027D
S12305008D05813B26E939860D8D09860A8D058D008D004F7EC0032F5E5E5E47524545548C
S1230520494E47532046524F4D204F5448454C4C4F2F444F20594F552057414E5420494E0B
S1230540535452554354494F4E533F3B2F2F4F5448454C4C4F20495320504C4159454420CF
S12305604F4E20414E2038204259203820434845434B455220424F415244205749544820A7
S12305802F524F5753204E554D4245524544203120544F203820414E4420434F4C554D4E1E
S12305A053204120544F20482E2F54484520494E495449414C20434F4E46494755524154DE
S12305C0494F4E20495320414C4C20424C414E4B204558434550542F464F522054484520D4
S12305E043454E54455220464F555220535155415245532C20574849434820464F524D2063
S1230600544845205041545445524E3A2F202020202020202020204F20582F202020202078
S1230620202020202058204F2F50555420594F555220504945434520534F205448415420FF
S12306404D494E45204953204245545745454E2032204F4620594F5552532C20535543483F
S12306602041533A2F202020202020202058204F20582F2020202020202020202058204FE4
S12306802F544849532057494C4C2022464C495022204D5920544F5020224F2220494E5471
S12306A04F20594F5552202258222F2F4E4F54453A20594F55204D415920434150545552DB
S12306C0452031204F52204D4F5245204F46204D5920504945434553205448495320574108
S12306E0592C2F4F5220594F55204D415920464F524645495420425920545950494E472078
S1230700225A222F2F53484F554C4420492057414954204245464F5245204D414B494E47A2
S1230720204D59204D4F5645533F3B2F4F4B2E20545950494E4720414E5920434841524152
S1230740435445522057494C4C204C4554204D4520474F212F3B2F53484F554C4420492090
S1230760504C4159204D5920424553542053545241544547593F3B2F534F5252592C2054B0
S123078048415420535155415245204953204F434355504945442E205452592041474149E0
S12307A04E213B2F594F5552204D4F56452D2D28524F572C434F4C293F3B2F444F20594F05
S12307C0552057414E5420544F20484156452058204F52204F3F3B2F444F20594F552057E7
S12307E0414E5420544F20474F2046495253543F3B2F534F5252592C20594F552041524568
S1230800204E4F54204E45585420544F204F4E45204F46204D59205049454345532E2054A9
S1230820525920414741494E213B2F534F5252592C2054484154204D4F564520444F455340
S1230840204E4F5420464C414E4B204120524F572E2054525920414741494E213B5E2F5474
S123086048415420474956455320594F55203B204F46204D59205049454345532F3B075963
S12308804F552048415645203B2050494543455320414E4420492048415645203B20504984
S12308A045434553212F3B534F5252592C204920574F4E2054484154204F4E45212F3B4122
S12308C020544945212F3B594F5520574F4E21212F3B54484154205741532041203B50453D
S12308E052464543542047414D45212F3B57414C4B41574159212F3B4649474854212F3BD2
S1230900484F542047414D45212F3B53515545414B4552212F3B2F444F20594F55205741A0
S12309204E5420544F20504C415920414E4F544845522047414D453F3B2F5448414E4B531B
S123094020464F5220504C4159494E47212F3B5E5E49204D4F564520544F203B2F54484147
S123096054204749564553204D45203B204F4620594F5552205049454345532E2F3B492076
S12309804841564520544F20464F52464954204D59204D4F5645212F3B2F41524520594F0B
S12309A05520464F5246454954494E4720594F5552205455524E202859204F52204E293FC1
S11809C03B2F20204120422043204420452046204720482F3B06
S9030100FB
